S01A000064656D6F70726F675F73746D3332663330332E7372656399
S3150800200000300020E1260008AD260008AF260008AB
S31508002010B1260008B3260008B5260008000000000F
S31508002020000000000000000000000000B7260008BD
S31508002030B926000800000000BB260008BD260008D7
S315080020403127000831270008312700083127000802
S3150800205031270008312700083127000831270008F2
S3150800206031270008312700083127000831270008E2
S3150800207031270008312700083127000831270008D2
S3150800208031270008312700083127000831270008C2
S3150800209031270008312700083127000831270008B2
S315080020A031270008312700083127000831270008A2
S315080020B031270008312700080000000031270008F2
S315080020C03127000800000000000000003127000842
S315080020D000000000312700083127000831270008D2
S315080020E03127000831270008000000000000000022
S315080020F000000000000000000000000000000000D2
S3150800210000000000000000000000000000000000C1
S3150800211000000000000000003127000831270008F1
S3150800212000000000000000000000000000000000A1
S315080021300000000000000000000000000000000091
S3150800214031270008312700080000000000000000C1
S315080021500000000000000000000000000000000071
S315080021600000000000000000000000000000000061
S315080021700000000000000000000000000000000051
S311080021800000000031270008EE11AA55E7
S3150800218C10B5054C237833B9044B13B10448AFF397
S3150800219C00800123237010BD0C00002000000000F5
S315080021AC283C000808B5034B1BB103490348AFF399
S315080021BC008008BD0000000010000020283C000824
S315080021CC08B500F06FF900F03DF900F0B1F808BD5C
S315080021DC08B500F041F900F02FF908BD08B5094813
S315080021EC094B03604FF46143436000238360C3606B
S315080021FC03610C2242618361C3610362436201F08D
S3150800220CB0FC08BD50000020004400402DE9F04108
S3150800221C04460D461746984601F014FA154BA3FBCF
S3150800222C00308009002201E00132D2B2112A1DD8F1
S3150800223C114B13F8121003EB420393F801C001EB90
S3150800224C0C0303FB0443B0FBF3FE03FB1E06002E34
S3150800225CEAD11FFA8EF32B80013B9BB2B3F5806F44
S3150800226CE2D2397088F800C0012000E00020BDE8F1
S3150800227CF08100BFD34D6210403C000870B58CB09D
S3150800228C0025ADF82E508DF82D500CAB03F8045DD7
S3150800229C0DF12D020DF12E014FF4FA70FFF7B6FF72
S315080022AC1A4C1B4B236025766576A5760126E676B1
S315080022BC25776577A560E5609DF82D30013B1B04F5
S315080022CC23619DF82C30013B1B056361BDF82E304C
S315080022DC6360204600F072FA0695079508964CF648
S315080022ECE043019302954FF6E0730393042304939A
S315080022FC059509960E230A9301A9204600F004FBBE
S3150800230C204600F07FFB0CB070BD00BF28000020F3
S3150800231C0064004008B5002301220146034801F079
S3150800232C5CFB08B1002008BD0120FCE7500000202A
S3150800233C08B5FFF753FFFFF7A1FF08BDBFF34F8F93
S3150800234C0549CA6802F4E062044B1343CB60BFF339
S3150800235C4F8F00BFFDE700BF00ED00E00400FA0553
S3150800236C08B5214B1B78B3B92048FFF7D3FF0128D2
S3150800237C00D008BD1D4B1B78013BDBB23F2BF8D8B0
S3150800238C00F091F81A4B1860174B01221A70194B6A
S3150800239C00221A70EDE7174B1B78013313481844C3
S315080023ACFFF7B8FF012813D1124A13780133DBB2B1
S315080023BC13700E4A12789342DBD10B4A0021117026
S315080023CC0A4A5278FF2AD4D1022BD2D1FFF7B6FF8C
S315080023DC00F069F8064B1B6864339842C9D9024B5E
S315080023EC00221A70C5E700BF11010020D00000209A
S315080023FC140100201201002000B58BB001AB03AA12
S3150800240C00210C4800F02CFB20B9039A40F26763B4
S3150800241C9A4202D00BB05DF804FB059B002BF9D150
S3150800242C9DF80430FF2BF5D1079B022BF2D1FFF751
S3150800243C85FF00BF2800002008B5FFF791FFFFF7BE
S3150800244CDBFF08BD08B500220821024800F0C2FCD3
S3150800245C08BD00BF0004004810B500F024F80E4B68
S3150800246C1B68C31AB3F5FA7F0CD304460B4B1B78BF
S3150800247C4BB90122094B1A700821094800F0AAFC2D
S3150800248C054B1C6010BD0022044B1A700821044829
S3150800249C00F0A0FCF4E700BF1C0100201801002086
S315080024AC00040048704708B500F082F908BD000022
S315080024BC014A024B9A6070470020000800ED00E0C4
S315080024CC30B589B0002403940494059406940794B3
S315080024DC164B5A6942F480025A615A6902F4800210
S315080024EC0092009A5A6942F400325A615A6902F407
S315080024FC00320192019A5A6942F480225A615B6948
S3150800250C03F480230293029B094D22460821284690
S3150800251C00F060FC082303930123049305940694A6
S3150800252C03A9284600F092FB09B030BD0010024002
S3150800253C0004004830B591B02022002107A801F00C
S3150800254C65FB0024019402940394049405940225D3
S3150800255C069501230A9310230B930D954FF46013DC
S3150800256C0F9306A800F03CFC0F23019302950394E5
S3150800257C4FF4806304930594294601A800F08AFF5A
S3150800258C11B030BD08B5FFF793FF00F0F3F8FFF76D
S3150800259CD1FFFFF795FFFFF713FEFFF719FEFCE7D0
S315080025AC82B00A4B9A6942F001029A619A6902F062
S315080025BC01020092009ADA6942F08052DA61DB690C
S315080025CC03F080530193019B02B070470010024040
S315080025DC00B589B0002303930493059306930793D8
S315080025EC0268144B9A4202D009B05DF804FB03F555
S315080025FCD633DA6942F00072DA61DA6902F00072EF
S3150800260C0192019A5A6942F400325A615B6903F4E1
S3150800261C00330293029B4FF4C05303930223049393
S3150800262C032306930923079303A94FF0904000F060
S3150800263C0DFBD9E70064004000B589B0002303936D
S3150800264C04930593069307930268144B9A4202D097
S3150800265C09B05DF804FB03F5E633DA6942F4003297
S3150800266CDA61DA6902F400320192019A5A6942F483
S3150800267C00325A615B6903F400330293029B48F2F9
S3150800268C0403039302230493032306930723079354
S3150800269C03A94FF0904000F0D9FAD9E7004400405E
S315080026AC7047FEE7FEE7FEE7FEE7704770477047A0
S315080026BC08B500F071F808BD054BD3F8882042F42C
S315080026CC7002C3F888204FF000629A60704700BF0A
S315080026DC00ED00E0DFF834D0002103E00C4B5B582A
S315080026EC435004310B480C4B42189A42F6D30B4A0A
S315080026FC02E0002342F8043B094B9A42F9D3FFF750
S3150800270CDBFF01F05FFAFFF73DFFFEE70030002024
S3150800271CA43C0008000000200C0000200C0000203F
S3150800272C24010020FEE7000010B504460E4B18786D
S3150800273C4FF47A73B3FBF0F30C4A1068B0FBF3F062
S3150800274C00F06EFA68B90F2C01D901200AE00022B4
S3150800275C21464FF0FF3000F02FFA054B1C60002085
S3150800276C00E0012010BD00BF04000020000000207E
S3150800277C0800002008B5074A136843F010031360D5
S3150800278C032000F007FA0020FFF7CEFFFFF708FF3B
S3150800279C002008BD00200240034A1168034B1B7831
S315080027AC0B441360704700BF200100200400002072
S315080027BC014B1868704700BF20010020002800F064
S315080027CCA18038B5044690F82030D3B12268136836
S315080027DC23F002031360FFF7EBFF054623685A68DC
S315080027EC12F0020F10D0FFF7E3FF401B0A28F5D9A9
S315080027FC636A43F400336362052384F820300120AE
S3150800280C38BDFFF7E5FEE1E71A6842F001021A60E7
S3150800281CFFF7CEFF054623685A6812F0010F0DD153
S3150800282CFFF7C6FF401B0A28F5D9636A43F4003341
S3150800283C6362052384F820300120E1E7227E012A11
S3150800284C3DD01A6822F080021A60637E012B3BD0B9
S3150800285C2268136823F040031360A37E012B39D03A
S3150800286C2268136823F020031360E37E012B37D00C
S3150800287C2268136843F010031360237F012B35D0AD
S3150800288C2268136823F008031360637F012B33D087
S3150800289C2268136823F004031360A368E2681343E1
S315080028AC22691343626913436268013A2168134328
S315080028BCCB6100206062012384F82030A0E71A68F7
S315080028CC42F080021A60C0E72268136843F040039E
S315080028DC1360C2E72268136843F020031360C4E749
S315080028EC2268136823F010031360C6E7226813687E
S315080028FC43F008031360C8E72268136843F004031F
S3150800290C1360CAE701207047036890F82020013A43
S3150800291CD2B2012A05D9436A43F4802343620120C3
S3150800292C704770B4D3F8002242F00102C3F80022B3
S3150800293C4A6902F01F02012000FA02F2D3F81C427F
S3150800294CD0430440C3F81C42CC69ACB9D3F80C424A
S3150800295C0440C3F80C42CE688D884C6945EA064596
S3150800296C483443F834508E680D884C6945EA064558
S3150800297C483403EBC4046560CC69012C19D08C6906
S3150800298C74BBD3F804420440C3F804420C696CBB0C
S3150800299CD3F814422040C3F81402096A01292BD033
S315080029ACD3F8002222F00102C3F80022002070BCE2
S315080029BC7047D3F80C421443C3F80C420E688D8842
S315080029CC4C6945EA0645483443F834508E688D8977
S315080029DC4C6945EA0645483403EBC4046560CEE702
S315080029ECD3F804421443C3F80442CFE7D3F81402CD
S315080029FC1043C3F81402D0E7D3F81C120A43C3F8E1
S31508002A0C1C22CDE738B590F82030DBB2012B05D067
S31508002A1C436A43F400234362012038BD044602236B
S31508002A2C80F820300268136823F001031360FFF75F
S31508002A3CBFFE054623685B6813F0010F0DD0FFF740
S31508002A4CB7FE401B0A28F5D9636A43F40033636260
S31508002A5C052384F820300120DFE700206062DCE7DC
S31508002A6C30B490F82040013CE4B2012C06D9436AF4
S31508002A7C43F480234362012030BC704700296FD190
S31508002A8C0468E46814F0030F64D0056801F11B04AC
S31508002A9C24012C5904F004049460002C6BD10568AD
S31508002AAC01F11B0424012C59640D1460056801F10D
S31508002ABC1B0424012D5905F00205D560056825442B
S31508002ACC6D6805F00F051561056825446D68C5F335
S31508002ADC0725956105682C446468240C54610468C0
S31508002AEC0A011444D4F8B8411C7004681444D4F888
S31508002AFCB841C4F307245C7004681444D4F8B8418C
S31508002B0CC4F307449C7004681444D4F8B841240EE2
S31508002B1CDC7004681444D4F8BC411C710468144471
S31508002B2CD4F8BC41C4F307245C7104681444D4F883
S31508002B3CBC41C4F307449C7104682244D2F8BC21F6
S31508002B4C120EDA71F9B90268D36843F02003D36020
S31508002B5C002091E7436A43F40013436201208BE794
S31508002B6C0468246914F0030F8FD1436A43F40013E5
S31508002B7C4362012080E7056801F11B0424012C59E6
S31508002B8CE408546092E70268136943F02003136162
S31508002B9C002071E7074AD36823F4E0631B041B0C77
S31508002BAC000200F4E060184340F0BF6040F40030C7
S31508002BBCD060704700ED00E030B4174BDB68C3F308
S31508002BCC0223C3F10704042C28BF04241D1D062D5B
S31508002BDC18D9033B4FF0FF3505FA04F421EA040132
S31508002BEC994005FA03F322EA0303194300280BDB81
S31508002BFC0901C9B200F1604000F5614080F8001384
S31508002C0C30BC70470023E5E700F00F000901C9B294
S31508002C1C024B1954F4E700BF00ED00E014ED00E098
S31508002C2C0138B0F1807F0AD2064B5860064AF0216B
S31508002C3C82F823100020986007221A60704701203A
S31508002C4C704700BF10E000E000ED00E0F0B583B07F
S31508002C5C002336E0032400E00024B4403C4302354C
S31508002C6C584E46F82540584C2568D44304EA0506C0
S31508002C7C4F6817F4803F01D042EA0506524D2E6084
S31508002C8C6D6804EA05064F6817F4003F01D042EA5E
S31508002C9C05064D4D6E60AD6804EA05064F6817F4D7
S31508002CAC801F01D042EA0506474DAE60ED682C4000
S31508002CBC4E6816F4001F01D042EA0504424AD46055
S31508002CCC01330A6832FA03F479D001249C40224075
S31508002CDCF6D04D686E1E012E03D9112D01D0122D7A
S31508002CEC12D186685F000325BD4026EA0506CD6825
S31508002CFCBD4035438560466826EA04064D68C5F32B
S31508002D0C00149C4034434460C5685F000324BC40EF
S31508002D1CE44325408E68BE402E43C6604D68022D9E
S31508002D2C01D0122D13D1DE08083650F826E003F030
S31508002D3C07054FEA850C0F2505FA0CF52EEA050E44
S31508002D4C0D6905FA0CF545EA0E0540F82650056896
S31508002D5C2C404D6805F00305BD402C4304604C68B7
S31508002D6C14F0805FACD0194CA56945F00105A56136
S31508002D7CA46904F001040194019C9D08AE1C114C35
S31508002D8C54F8267003F00304A6000F24B44027EA6F
S31508002D9C0407B0F1904F3FF45FAF0D4CA0420AD038
S31508002DAC04F58064A04208D004F58064A0423FF480
S31508002DBC51AF052451E701244FE702244DE703B030
S31508002DCCF0BD00BF000001400004014000100240A5
S31508002DDC000400480AB98162704781617047000097
S31508002DEC002800F00D8370B582B00446036813F012
S31508002DFC010F3BD0B54B5B6803F00C03042B1ED0BC
S31508002E0CB24B5B6803F00C03082B13D06368B3F55D
S31508002E1C803F68D0002B40F0928003F1804303F585
S31508002E2C04331A6822F480321A601A6822F4802253
S31508002E3C1A605DE0A54B5B6813F4803FE6D04FF44F
S31508002E4C003393FAA3F3A14B19684FF4003393FAA2
S31508002E5CA3F3B3FA83F303F01F03012202FA03F375
S31508002E6C0B4203D06368002B00F0CC82236813F066
S31508002E7C020F00F0C680954B5B6813F00C0F00F040
S31508002E8C9C80924B5B6803F00C03082B00F08F8038
S31508002E9C2369002B00F0F380012292FAA2F3B3FA0D
S31508002EAC83F303F1845303F584139B001A60FFF72D
S31508002EBC7FFC0546022393FAA3F3844B1968022375
S31508002ECC93FAA3F3B3FA83F303F01F03012202FA6E
S31508002EDC03F30B4240F0C480FFF76AFC401B022840
S31508002EECE8D9032095E2794A136843F480331360D2
S31508002EFC764AD36A23F00F03A1680B43D36263683F
S31508002F0C002B36D0FFF754FC05464FF4003393FAE2
S31508002F1CA3F36E4B19684FF4003393FAA3F3B3FA81
S31508002F2C83F303F01F03012202FA03F30B429DD12C
S31508002F3CFFF73EFC401B6428E7D9032069E2B3F58A
S31508002F4CA02F09D0614B1A6822F480321A601A68CD
S31508002F5C22F480221A60CBE703F18043A3F53C33B5
S31508002F6C1A6842F480221A601A6842F480321A608F
S31508002F7CBEE7FFF71DFC05464FF4003393FAA3F39F
S31508002F8C524B19684FF4003393FAA3F3B3FA83F34D
S31508002F9C03F01F03012202FA03F30B423FF466AF58
S31508002FACFFF706FC401B6428E6D9032031E2474BA1
S31508002FBC5B6813F4803F7FF46BAF022393FAA3F399
S31508002FCC424B1968022393FAA3F3B3FA83F303F07B
S31508002FDC1F03012202FA03F30B4204D0236993421E
S31508002FEC01D0012015E23948036823F0F80361691A
S31508002FFCF82292FAA2F2B2FA82F201FA02F2134318
S3150800300C0360236813F0080F00F08C80A369002B6B
S3150800301C60D0012191FAA1F2B2FA82F22C4B134438
S3150800302C9B001960FFF7C4FB0546022393FAA3F22B
S3150800303C93FAA3F293FAA3F2244A516A93FAA3F3E6
S3150800304CB3FA83F303F01F03012202FA03F30B42CC
S3150800305C68D1FFF7ADFB401B0228E6D90320D8E15F
S3150800306C1A48036823F0F8036169F82292FAA2F267
S3150800307CB2FA82F201FA02F213430360C1E70123A2
S3150800308C93FAA3F3B3FA83F303F1845303F5841386
S3150800309C9B0000221A60FFF78BFB0546022393FA66
S315080030ACA3F30A4B1968022393FAA3F3B3FA83F32F
S315080030BC03F01F03012202FA03F30B42A1D0FFF718
S315080030CC77FB401B0228E9D90320A2E10010024035
S315080030DC20819010012292FAA2F2B2FA82F2BC4B2B
S315080030EC13449B0000221A60FFF762FB0546022375
S315080030FC93FAA3F293FAA3F293FAA3F2B54A516A96
S3150800310C93FAA3F3B3FA83F303F01F03012202FA2B
S3150800311C03F30B4206D0FFF74BFB401B0228E6D9FC
S3150800312C032076E1236813F0040F00F0B380A94B53
S3150800313CDB6913F0805F20D1A64BDA6942F0805226
S3150800314CDA61DB6903F080530193019B0125A24BDD
S3150800315C1B6813F4807F12D0E368012B23D073BB52
S3150800316C03F1804303F504331A6A22F001021A624A
S3150800317C1A6A22F004021A621AE00025E7E7964A50
S3150800318C136843F480731360FFF712FB0646924BE1
S3150800319C1B6813F4807FDFD1FFF70AFB801B6428BA
S315080031ACF5D9032035E18B4A136A43F00103136200
S315080031BCE368002B41D0FFF7FBFA06462BE0052BFC
S315080031CC09D0844B1A6A22F001021A621A6A22F092
S315080031DC04021A62ECE77F4B1A6A42F004021A627E
S315080031EC1A6A42F001021A62E2E77A4B196A02235A
S315080031FC93FAA3F3B3FA83F303F01F03012202FA3B
S3150800320C03F3194245D1FFF7D3FA801B41F28833F1
S3150800321C984200F2F980022393FAA3F293FAA3F3E5
S3150800322CB3FA83F35B0943F00203022BDDD00223C6
S3150800323C93FAA3F3674B596AD9E7FFF7B9FA064627
S3150800324C15E0644B196A022393FAA3F3B3FA83F3D2
S3150800325C03F01F03012202FA03F3194219D0FFF7F0
S3150800326CA7FA801B41F28833984200F2CF800223DA
S3150800327C93FAA3F293FAA3F3B3FA83F35B0943F035
S3150800328C0203022BDDD0022393FAA3F3514B596A9E
S3150800329CD9E7B5BBE369002B00F0BA804D4A5268F2
S315080032AC02F00C02082A00F09980022B2FD04FF05E
S315080032BC807393FAA3F3B3FA83F303F1845303F5F8
S315080032CC84139B0000221A60FFF772FA04464FF02B
S315080032DC007393FAA3F33F4B19684FF0007393FAF4
S315080032ECA3F3B3FA83F303F01F03012202FA03F3E1
S315080032FC19426BD0FFF75CFA001B0228E7D90320AA
S3150800330C87E0344AD36923F08053D361C2E74FF080
S3150800331C807393FAA3F3B3FA83F303F1845303F597
S3150800332C84139B0000221A60FFF742FA05464FF0F9
S3150800333C007393FAA3F3274B19684FF0007393FAAB
S3150800334CA3F3B3FA83F303F01F03012202FA03F380
S3150800335C194206D0FFF72CFA401B0228E7D903209E
S3150800336C57E01C494B6823F47413626A206A0243BB
S3150800337C13434B604FF0807393FAA3F3B3FA83F3BA
S3150800338C03F1845303F584139B0001221A60FFF79B
S3150800339C0FFA04464FF0007393FAA3F30D4B196812
S315080033AC4FF0007393FAA3F3B3FA83F303F01F03F6
S315080033BC012202FA03F3194206D1FFF7F9F9001BA9
S315080033CC0228E7D9032024E0002022E0002020E090
S315080033DC208190100010024000700040012B1AD07A
S315080033EC0F4B5B6803F48031226A914201D00120AD
S315080033FC0FE003F47013626A93420ED0012008E0C2
S3150800340C01207047012004E0032002E0032000E0BD
S3150800341C002002B070BD0120FBE70020F9E700BFD1
S3150800342C00100240164B596801F00C03082B24D1E6
S3150800343C01F470124FF4701393FAA3F3B3FA83F3EF
S3150800344C22FA03F30F4AD05C0D4BDB6A03F00F0329
S3150800345C0F2292FAA2F2B2FA82F2D3400A4AD25C4C
S3150800346C11F4803F03D1094B03FB00F07047084B5E
S3150800347CB3FBF2F300FB03F070470548704700BF37
S3150800348C001002407C3C00088C3C000800093D00FA
S3150800349C00127A00002800F0C18070B50446614B12
S315080034AC1B6803F007038B420CD25E4A136823F0A1
S315080034BC07030B431360136803F007038B4201D011
S315080034CC012070BD236813F0020F06D0564A5368C4
S315080034DC23F0F003A068034353600D46236813F0EA
S315080034EC010F5AD06368012B2DD0022B40D0022233
S315080034FC92FAA2F24C4A1068022292FAA2F2B2FA94
S3150800350C82F202F01F02012101FA02F2104200F0C7
S3150800351C878045494A6822F0030213434B60FFF73C
S3150800352C47F90646404B5B6803F00C036268B3EB3D
S3150800353C820F32D0FFF73CF9801B41F28833984250
S3150800354CF0D90320BDE74FF4003292FAA2F2364ABC
S3150800355C10684FF4003292FAA2F2B2FA82F202F032
S3150800356C1F02012101FA02F20242D2D10120A8E778
S3150800357C4FF0007292FAA2F22B4A10684FF00072C2
S3150800358C92FAA2F2B2FA82F202F01F02012101FAB1
S3150800359C02F21042BDD1012093E7224B1B6803F0BF
S315080035AC0703AB420CD91F4A136823F007032B43B6
S315080035BC1360136803F00703AB4201D0012080E7C0
S315080035CC236813F0040F06D0174A536823F4E063F4
S315080035DCE1680B435360236813F0080F07D0124AAF
S315080035EC536823F46053216943EAC1035360FFF718
S315080035FC19FF0D4B5B6803F0F003F02292FAA2F266
S3150800360CB2FA82F2D340094AD35CD840084B186008
S3150800361C084B1868FFF788F8002052E70120704716
S3150800362C01204EE70020024000100240643C0008CE
S3150800363C0000002008000020014B1868704700BFE6
S3150800364C0000002008B5FFF7F7FF074B5B6803F48B
S3150800365CE0634FF4E06292FAA2F2B2FA82F2D34035
S3150800366C024AD35CD84008BD00100240743C0008DE
S3150800367C08B5FFF7E1FF074B5B6803F460534FF49B
S3150800368C605292FAA2F2B2FA82F2D340024AD35CA0
S3150800369CD84008BD00100240743C000810B504461A
S315080036AC83680269134342691343C2691343016869
S315080036BC08686C4A024013430B602268536823F46B
S315080036CC4053E1680B435360A269236A1A43216885
S315080036DC8B6823F4306313438B602368624A9342E6
S315080036EC15D0624A934228D002F58062934220D0C4
S315080036FC1023E269B2F5004F21D0082B00F2AB80FB
S3150800370CDFE803F06C818BA996A9A9A9A000584BF0
S3150800371C1B6B03F00303032B09D8DFE803F0020441
S3150800372C060C0023E5E70423E3E70823E1E7102367
S3150800373CDFE70023DDE70223DBE70023D9E7082BC5
S3150800374C49D8DFE803F0051E2948344848483F00A5
S3150800375CFFF778FF6268530803EB4003B3FBF2F3F9
S3150800376C9BB20020A3F110014FF6EF72914275D867
S3150800377C9AB222F00F02C3F3420313432268D360B2
S3150800378C3DE0FFF775FF6268530803EB4003B3FB94
S3150800379CF2F39BB20020E5E76268530803F574035D
S315080037AC03F51053B3FBF2F39BB20020DAE7FFF7ED
S315080037BC39FE6268530803EB4003B3FBF2F39BB282
S315080037CC0020CFE76268530803F58033B3FBF2F3A6
S315080037DC9BB20020C6E701200023C3E7FFF732FFA0
S315080037EC626800EB5203B3FBF2F39BB20020A3F121
S315080037FC10014FF6EF72914232D82268D36000233B
S3150800380C2366636610BDFFF733FF626800EB52034D
S3150800381CB3FBF2F39BB20020E9E76268530803F5A1
S3150800382CF40303F59053B3FBF2F39BB20020DEE7E7
S3150800383CFFF7F8FD626800EB5203B3FBF2F39BB299
S3150800384C0020D4E76268530803F50043B3FBF2F390
S3150800385C9BB20020CBE701200023C8E70120CEE766
S3150800386C0120CCE7F369FFEF003801400044004023
S3150800387C00100240436A13F0010F06D00268536821
S3150800388C23F40033816A0B435360436A13F0020F27
S3150800389C06D00268536823F48033C16A0B4353601D
S315080038AC436A13F0040F06D00268536823F4802386
S315080038BC016B0B435360436A13F0080F06D002687A
S315080038CC536823F40043416B0B435360436A13F06C
S315080038DC100F06D00268936823F48053816B0B4350
S315080038EC9360436A13F0200F06D00268936823F49A
S315080038FC0053C16B0B439360436A13F0400F0AD015
S3150800390C0268536823F48013016C0B435360036CF1
S3150800391CB3F5801F0BD0436A13F0800F06D00268EC
S3150800392C536823F40023816C0B4353607047026879
S3150800393C536823F4C003416C0B435360EBE72DE942
S3150800394CF04104460F4616469846069D2368DB69E1
S3150800395C37EA03030CBF01230023B3423AD1B5F16E
S3150800396CFF3FF3D0FEF724FFA0EB0800A8421FD8B0
S3150800397CF5B123681A6812F0040FE7D0DA6912F465
S3150800398C006FE3D04FF400621A622268136823F4BE
S3150800399CD07313602268936823F001039360202385
S315080039AC6367A367E367002384F87030032012E08B
S315080039BC2268136823F4D07313602268936823F083
S315080039CC0103936020236367A367002384F8703090
S315080039DC032000E00020BDE8F0812DE9F04383B018
S315080039EC1E46836F202B7AD104460D469046002935
S315080039FC79D0002A79D090F87030012B77D0012332
S31508003A0C80F870300023C36722238367FEF7D0FE45
S31508003A1C0746A4F85880A4F85A80A368B3F5805FC3
S31508003A2C06D0A3B9226972B9FF22A4F85C2014E067
S31508003A3C226922B940F2FF12A4F85C200DE0FF229D
S31508003A4CA4F85C2009E07F22A4F85C2005E0B3F119
S31508003A5C805F0AD00022A4F85C20B4F85C80B3F529
S31508003A6C805F0CD04FF000091DE022691AB97F223D
S31508003A7CA4F85C20F1E73F22A4F85C20EDE7236963
S31508003A8C13B14FF000090EE0A94600250BE0236898
S31508003A9C9B8C08EA030329F8023BB4F85A30013B1D
S31508003AAC9BB2A4F85A30B4F85A309BB28BB1009634
S31508003ABC3B46002220212046FFF741FFC8B9002DBE
S31508003ACCE5D023689A8C5FFA88F3134005F8013B16
S31508003ADCE3E72023A367002084F8700000E00220A7
S31508003AEC03B0BDE8F0830120FAE70120F8E70220CD
S31508003AFCF6E70320F4E730B583B004460023C36722
S31508003B0CFEF756FE054623681B6813F0080F0CD102
S31508003B1C23681B6813F0040F15D120236367A3676A
S31508003B2C002084F8700003B030BD6FF07E4300931C
S31508003B3C034600224FF400112046FFF700FF002829
S31508003B4CE6D00320EFE76FF07E4300932B46002266
S31508003B5C4FF480012046FFF7F2FE0028DDD0032043
S31508003B6CE1E768B310B50446436F03B324236367D0
S31508003B7C2268136823F0010313602046FFF78EFDB5
S31508003B8C012813D0636ABBB92268536823F490439F
S31508003B9C53602268936823F02A039360226813689B
S31508003BAC43F0010313602046FFF7A5FF10BD80F80C
S31508003BBC7030FEF741FDD9E72046FFF75BFEE3E7D9
S31508003BCC0120704770B50D4E0D4CA41BA410002592
S31508003BDCA54209D10B4E0C4C00F020F8A41BA410DE
S31508003BEC0025A54205D170BD56F8253098470135F4
S31508003BFCEEE756F8253098470135F2E79C3C000865
S31508003C0C9C3C00089C3C0008A03C00080244034667
S31508003C1C934200D1704703F8011BF9E7F8B500BFCA
S31508003C2CF8BC08BC9E467047F8B500BFF8BC08BC83
S30908003C3C9E467047DB
S31508003C4005020602060307030803090309040A0412
S31508003C500B040C040C050D050E050F050F061006C2
S31508003C60100710080000000000000000010203040D
S31508003C700607080900000000010203040203040500
S31508003C80060708090A0B0C0D0E0F10100102030493
S31108003C9005060708090A0B0C0D0E0F109C
S30908003C9CB12100083C
S30908003CA08D2100085C
S31108003CA400127A00010000001000000069
S705080026E1EB
